:020000020000FC
:1000000000C00FE50DBF08E00EBF0FEF01BB07BB3F
:100010000ABB02BB0BBB0CE000B938D050EA3ED0A3
:1000200010E046D020E049D011E042D020E045D099
:1000300012E03ED020E041D013E03AD020E33DD0A2
:1000400014E036D029E039D015E032D029EE35D091
:1000500016E02ED026E631D039D03FD050EA10E05D
:1000600020E014D01BD024D028D030D036D050EA95
:1000700061EA12E00BD012D01BD00CD014D022D0E9
:1000800025D02BD023B1209528BBF1CF04EA06BFA1
:1000900020D0089504EA06BF1CD0089553B904E89F
:1000A00006BF17D0089563B904E806BF12D00895BB
:1000B00013B904E806BF0DD0089523B904E806BFBC
:1000C00008D0089504E806BF04D0089504E906BFE7
:1000D000089506B707FFFDCF08957FEF84E38A9563
:0800E000F1F77A95D9F70895B4
:00000001FF
